:1000000012C05DC52AC029C0C3C5C5C426C025C04D
:10001000B1C4F8C322C0EFC220C0BCC21EC01DC004
:10002000C1C561C51AC011241FBECFE5D4E0DEBF33
:10003000CDBF10E0A0E6B0E0E8EBF1E102C0059032
:100040000D92A037B107D9F713E0A0E7B0E001C0E7
:100050001D92A339B107E1F73AC1D2CF20918200B6
:1000600080916100821710F4282FAB9A8091800054
:10007000909181008338910560F01BBC1ABC19BCBB
:1000800018BC13BCAB9A01979093810080938000B9
:100090000895822F9927880F991F9BBD8ABD99BD0E
:1000A00088BD23BD089582E08FBD81E485BD85B301
:1000B000817F85BB89E08EBD089592B7980F82B786
:1000C000891B87FDFCCF0895AF92BF92CF92DF923C
:1000D000EF92FF920F931F93CF93DF93182F8CE231
:1000E000A82E81E0B82EC12CD12C109297004398F5
:1000F00085E090E09093830080938200AFDF57D635
:1001000088EC90E0DDD3C12FDD27D0938300C0932E
:100110008200EE24FF248701EA14FB040C051D0570
:1001200078F480916600882311F43ED201C050D348
:1001300084E6C3DF0894E11CF11C011D111DECCF06
:10014000C601B5012FE030E040E050E013D8A21A1C
:10015000B30AC40AD50A0894A108B108C108D10895
:1001600089E1A816B104C104D104C8F020D6809159
:1001700099008F5F809399008091990066E0DAD7AB
:1001800090939900AED3D0938300C093820066DF32
:10019000449BBFCF82B390E8892782BBBACFDF915F
:1001A000CF911F910F91FF90EF90DF90CF90BF9074
:1001B000AF90089540917A0050917B004115510510
:1001C00009F04BC080917900882371F090918800EC
:1001D0008FEF989FC001112468EC70E0B7D770933F
:1001E00085006093840041C080918E00882341F196
:1001F000209190003091910081E02D32380708F075
:100200009A01293C310510F028EC30E02B30310503
:1002100028F4509385004093840026C08CEF90E032
:10022000289FA001299F500D389F500D1124CA010D
:10023000885D994064EB70E089D7CB01039610C0CC
:100240008091840090918500009729F00197909308
:10025000850080938400AB9A08C080918803992719
:100260009093850080938400AB9880918400909156
:1002700085008F3F910539F030F08FEF90E090933B
:10028000850080938400809184009927089580914F
:100290008000909181009093780380937703809100
:1002A0007E00992790937A03809379038091700060
:1002B0009091710090937C0380937B0380919000D8
:1002C0009091910090937E0380937D030895CFE5F4
:1002D000D4E0DEBFCDBFEE2488E084BB85BB8AEBD3
:1002E00081BB80E882BB8EE087BB81E388BB5BD2A9
:1002F000CAD27894C0E0D0E0C430D10509F4979A0E
:1003000086E990E0DDD297988AEF90E0D9D22196E5
:10031000C530D1058CF384EF91E0D2D244D2C3DE54
:1003200080E5DCD31AD385E690E0B6D286E690E08D
:10033000B3D287E690E0B0D2EC018EEF90E0ACD281
:100340005C018DEE93E0A8D28C018EEE93E0A4D2F6
:100350006C01CE01AAD28823E1F3979A1092830010
:10036000109282007BDE88E080BF81E087B98AE05E
:1003700090E092D2EC0181E090E090937A03809338
:100380007903109291001092900014DF99279093B6
:10039000830080938200809199008E1551F0109215
:1003A00062001092630082E390E076D2EC01E0906C
:1003B00099008091820090918300892BC9F410925A
:1003C000740010926300C80170D28823D9F0109293
:1003D0009700439881E08093620082B3877C82BB60
:1003E00082E08FBD81E485BD85B3817F85BB0AC076
:1003F00080916200882319F081E0809374008CED75
:1004000095E04AD280916200882321F01092830007
:100410001092820023DE809163008F5F80936300DF
:10042000813009F0B2CF809162008111979AC501A5
:100430003CD2882339F182E390E02ED25C01809196
:100440007E00482F5527209180003091810042176F
:10045000530710F48F5F04C02417350718F4815038
:1004600080937E0080917E0090916100823428F01C
:10047000915090936100AB9A05C09F3F19F09F5F28
:1004800090936100C80111D2882319F18AE090E0AD
:1004900003D28C012091720030917300C901880F42
:1004A000991F880F991F820F931F820F931F66E079
:1004B00070E04CD6709371006093700010927300DE
:1004C0001092720080918E00882319F481E080934D
:1004D0006000C601EAD1882321F08CED95E0DCD1E3
:1004E0006C01CE01E2D1882331F0809170009091AF
:1004F0007100892B29F080917400882309F445CF7D
:1005000021E0F22EF092620010929700439884E668
:1005100090E0C2D1EC0180917400882309F435CFBA
:10052000AB98109274008AE0CFDD979A1092620027
:100530008091990081508093990081E090E09093A0
:100540008300809382008ADD88B18C7F88B9F09225
:10055000970088B18A6088B984E690E09DD1EC016B
:10056000CE01A3D18823E1F38AE090E09093830049
:100570008093820073DD88EC90E08ED1EC01CE0197
:1005800094D18823E1F388EE93E086D1EC0197E0E3
:10059000E92EFBCE1F920F920FB60F9211240F90EF
:1005A0000FBE0F901F9018955E9B24C0809166002F
:1005B0008823E1F48091890090918A0001969093BC
:1005C0008A0080938900FC01E556FD4FE081ED3003
:1005D00019F08436910539F410928A00109289003E
:1005E00081E080936600589AECB9089510928A00D1
:1005F0001092890008951F920F920FB60F92112446
:100600008F938CB18093870080918700853F19F488
:100610001092670014C0809167008F5F809367001D
:10062000843041F4809187008093880088EC809327
:10063000790005C0853618F084E6809367008F91B5
:100640000F900FBE0F901F901895AC01A0E0B0E086
:100650009D01A817B90748F4EBE9F2E08191280F52
:10066000311D1196A417B507C8F33F70FD01E5567B
:10067000FD4FC90146E0969587954A95E1F7835C61
:1006800080831196FD01E556FD4F2F733070822F48
:10069000835C8083A456BD4F8DE08C9310926600DE
:1006A00080919B028CB908951F93CF93DF93382FCD
:1006B000EA01722F10E083E280939B0260939C0218
:1006C00030939D02A3E0B0E0772309F458C077236C
:1006D00011F4972F07C0FE01E10FF11D1F5F9081FC
:1006E000715011F4472F0EC0FE01E10FF11D1F5F85
:1006F0004081715039F0FE01E10FF11D1F5F6081F3
:10070000715001C0672FFD01E556FD4F892F869579
:100710008695835C80831196FD01E556FD4F892FF8
:1007200099278370907024E0880F991F2A95E1F72C
:1007300055279A0194E0369527959A95E1F7822BF3
:10074000835C80831196FD01E556FD4F4F7050701C
:10075000440F551F440F551F862F992756E0969535
:1007600087955A95E1F7842B835C80831196FD0170
:10077000E556FD4F6F73635C60831196A5CFCD0185
:1007800064DFDF91CF911F910895CF93C82F8A30F6
:1007900011F48DE0FADF5D9BFECFCCB980E090E0F4
:1007A000CF910895089588E18AB9599A579A89E1B5
:1007B00089B960E070E085EC93E05FD388EC90E06D
:1007C0006BD0909300038093FF028AE28CB9089566
:1007D0008091FF029091000368D0882391F080916E
:1007E0006600882371F022E245E653E060919A02A8
:1007F00084E45ADF82E390E04FD09093000380932B
:10080000FF0208951F920F920FB60F9211248F933B
:100810009F93809187038F5F8093870380918D00E2
:10082000815080938D008F3F39F583E080938D0058
:1008300080918B0090918C00019690938C00809316
:100840008B0080917A0090917B00009729F00197AE
:1008500090937B0080937A0080918E00882329F00A
:1008600080918E00815080938E0080917900882342
:1008700019F08150809379009F918F910F900FBE56
:100880000F901F90189582E083BF89B7816089BF60
:1008900089B7806489BF089520918B0030918C00C6
:1008A000280F391FC9010197089520918B003091BD
:1008B0008C00821B930B892F9927807899270895A4
:1008C000CF93DF93E9DFEC01CE01EFDF8823E1F383
:1008D000DF91CF91089586EA86B987E087B9369A85
:1008E000089527B196E097B910BE83ED86B9349A82
:1008F00097B9369A349BFECF27B944B155B1440F0E
:10090000551F440F551F493C510510F048EC50E06D
:100910002091800030918100C90163E0880F991F08
:100920006A95E1F7821B930B840F951F23E0969540
:1009300087952A95E1F7909381008093800020911C
:100940007F0033272817390720F480918000809397
:100950007F0016B888E080BF08958EB5806C8EBD8C
:100960008EB580648EBD89B7806289BF89B7846087
:1009700089BF08951F920F920FB60F9211248F9383
:1009800080918F008F5F80938F008F910F900FBEAB
:100990000F901F9018951F920F920FB60F9211246F
:1009A0002F933F938F939F930EB406FE0FC0109228
:1009B0008F0086B597B590939300809392008EB583
:1009C0008F7B8EBD84E680938E0070C08EB5806470
:1009D0008EBD26B537B58091920090919300281B6B
:1009E000390B80918F009927982F8827990F280F0E
:1009F000391F689414F8369527951694E1F73093CB
:100A00009500209394002851314030F488E191E022
:100A100090939500809394002091940030919500DC
:100A2000285131403093950020939400809190009C
:100A3000909191008217930730F4809190009091EB
:100A4000910001960CC08091900090919100281720
:100A5000390748F48091900090919100019790930C
:100A60009100809390002091900030919100C901F5
:100A7000880F991F880F991F880F991F821B930B4E
:100A80002091940030919500820F931F23E096955A
:100A900087952A95E1F79093950080939400909321
:100AA00091008093900081E0809360009F918F91EE
:100AB0003F912F910F900FBE0F901F9018951F928E
:100AC0000F920FB60F9211248F938AB78F7B8ABF34
:100AD0008F910F900FBE0F901F901895885F82B96D
:100AE00085EC86BF08951F920F920FB60F921124C6
:100AF0008F939F9381B19927887F9070803891055B
:100B0000E9F08138910534F40097B1F18036910510
:100B100079F035C0883B9105D9F0893B910524F4E3
:100B2000883A9105A9F02BC0883F910511F127C0A3
:100B300086B7806886BF1092960023C083B18093E9
:100B4000880384EF91E090937B0080937A000EC03D
:100B500090919600992339F480917E0083B99F5F2C
:100B60009093960003C08091610083B986B7806836
:100B700007C086B7806986BF86B7806986BF85EC67
:100B800086BF9F918F910F900FBE0F901F90189569
:100B90001F920F920FB60F9211240F900FBE0F905D
:100BA0001F9018951F920F920FB60F9211241F934A
:100BB0002F933F934F935F936F937F938F939F9365
:100BC000AF93BF93CF93EF93FF93459B02C011E088
:100BD00001C010E08091990099278230910509F4B5
:100BE00050C0833091052CF4009779F0019739F1CA
:100BF000BFC08430910509F478C0843091050CF4AD
:100C00005AC0059709F48BC0B3C082EA8FBD81E654
:100C100085BD88E087BB112369F082B3877E82BBE4
:100C2000959AC1E0C4BD8091600081115ADE409860
:100C3000C7B91BC082B3877D82BB949A99C082B327
:100C4000877E82BB959A1123B1F482EA8FBD81E43D
:100C500085BD8CE087BB81E084BD809160008111FF
:100C600040DE17B988B1836088B9809199008F5FA1
:100C7000809399006DC082EA8FBD81E685BD88E0D2
:100C800076C082EA8FBD81E485BD8CE087BB1123ED
:100C900069F082B38F7C82BB939A81E084BD80919E
:100CA000600081111EDE82E087B932C082B3877E88
:100CB00082BB959A5DC082B38F7C82BB939A1123CD
:100CC00071F482EA8FBD81E485BD8AE087BBC1E013
:100CD000C4BD80916000811104DEC7B9C3CF82EA30
:100CE0008FBD81E485BD8CE042C082EA8FBD81E486
:100CF00085BD8AE087BB112369F082B3877D82BB03
:100D0000949A81E084BD809160008111EADD17B87A
:100D10004098ABCF82B38F7C82BB939A29C082B3B9
:100D2000877D82BB949A1123E9F482EA8FBD81E624
:100D300085BD88E087BB81E084BD80916000811122
:100D4000D0DD82E087B988B1836088B910939900BB
:100D5000809172009091730001969093730080933C
:100D6000720006C082EA8FBD81E485BD8AE087BB40
:100D7000459903C0112309F028CF459B03C01123D7
:100D800009F423CF10926000FF91EF91CF91BF91B2
:100D9000AF919F918F917F916F915F914F913F9113
:100DA0002F911F910F900FBE0F901F90189580915B
:100DB000990099278230910551F1833091052CF4E7
:100DC000009769F00197B9F0089584309105E1F139
:100DD000843091055CF1059709F443C0089582EAD7
:100DE0008FBD81E685BD88E087BB82B3877D82BBEE
:100DF000949A82E034C082EA8FBD81E685BD88E0A6
:100E000087BB82B3877E82BB959A81E01AC082EA53
:100E10008FBD81E485BD8CE087BB82B3877E82BBBA
:100E2000959A17B888B1836088B9089582EA8FBD12
:100E300081E485BD8CE087BB82B38F7C82BB939AB3
:100E400082E087B94098089582EA8FBD81E485BD2C
:100E50008AE087BB82B38F7C82BB939A81E087B99B
:100E6000E1CF82EA8FBD81E485BD8AE087BB82B392
:100E7000877D82BB949A17B8E5CF0F931F93CF93CA
:100E8000DF938C01EB01009711F4672BB9F16EE051
:100E900070E081E090E037D0FC01892B71F180E8AF
:100EA0008383209771F0D387C28781E88383809101
:100EB000890390918A03892B21F4F0938A03E093AC
:100EC000890301151105C9F01187008783818260AC
:100ED000838380918B0390918C03892B71F4F09321
:100EE0008C03E0938B0380918D0390918E03892B6B
:100EF00021F4F0938E03E0938D03CF01DF91CF9126
:100F00001F910F9108950F931F93CF93DF93869FA7
:100F10008001879F100D969F100D1124C8010DD0E0
:100F2000EC01009721F0A80160E070E0FCD0CE0158
:100F3000DF91CF911F910F910895CF93DF93AC0173
:100F4000029710F442E050E020E030E0A0919103DD
:100F5000B0919203BD01F901109709F44CC08D9135
:100F60009C9111978417950731F14817590738F468
:100F70002115310519F08217930708F49C01FD0132
:100F8000A281B381109759F721153105A1F1C9014B
:100F9000841B950B049708F4A901DB01E0E0F0E065
:100FA000109749F18D919C91119782179307F9F44D
:100FB0004217530779F4ED018A819B81309719F02C
:100FC0009383828304C09093920380939103CD0115
:100FD00002964AC0241B350BFD01E20FF31F41931B
:100FE0005193225030402D933C93CF013DC0FD01E1
:100FF000A281B381D5CF80918F0390919003892BEB
:1010000041F480916B0090916C00909390038093D9
:101010008F03E0916900F0916A00309741F4EDB7D9
:10102000FEB780916D0090916E00E81BF90BA091C6
:101030008F03B09190039F012A1B3B0B24173507A8
:1010400088F0CA0102962817390760F0CD01840F95
:10105000951F02969093900380938F034D935D9319
:10106000CD0102C080E090E0DF91CF910895CF9351
:10107000DF93009709F454C0DC011297ED011B8245
:101080001A828091910390919203009721F1FC01C3
:1010900040E050E0EA17FB0718F1ED01FB83EA831B
:1010A0002D913C911197C20FD31FCE0102968E173E
:1010B0009F0771F48A819B81280F391F2E5F3F4F54
:1010C00011963C932E9382819381FD0193838283B9
:1010D0004115510559F4B0939203A093910320C098
:1010E000AF010280F381E02D3097A1F6EA01BB83C6
:1010F000AA83CA01029628813981820F931F8A1719
:101100009B0771F48D919C911197280F391F2E5FC9
:101110003F4F39832883FD01828193819B838A839A
:10112000DF91CF910895DC0101C06D934150504093
:10113000E0F70895991B79E004C0991F961708F00D
:10114000961B881F7A95C9F780950895AA1BBB1B2B
:1011500051E107C0AA1FBB1FA617B70710F0A61BB7
:10116000B70B881F991F5A95A9F780959095BC01D8
:10117000CD010895A1E21A2EAA1BBB1BFD010DC0D3
:10118000AA1FBB1FEE1FFF1FA217B307E407F50737
:1011900020F0A21BB30BE40BF50B661F771F881F13
:1011A000991F1A9469F760957095809590959B01A9
:0811B000AC01BD01CF0108955F
:1011B80001FF01010A00016464000093032000009C
:00000001FF
